:020000020000FC
:1000000014C0189518951895189518951895189561
:100010001895189518951895189518951895189578
:100020001895189518951895189500E806BD00E0E4
:1000300006BD00E00BBB03E00ABB00E808BB0FE70E
:1000400007BB0FE702BB0FE301BB0FED0DBFA89588
:1000500008E101BD0AE001BDA89500E808B9B8C2F1
:1000600003E10A95F1F708950D91013027950D915F
:10007000013027950D91013027950D91013027957D
:100080000D91013027950D91013027950D9101308B
:100090002795A7502695209528BB0D9102302795CE
:1000A0000D91023027950D91023027950D91023068
:1000B00027950D91023027950D91023027950D91CE
:1000C00002302795A7502695209528BBC9DF0D91B2
:1000D000033027950D91033027950D910330279517
:1000E0000D91033027950D91033027950D91033025
:1000F00027950D9103302795A7502695209528BB6D
:10010000AFDFAEDF0D91043027950D9104302795B8
:100110000D91043027950D91043027950D910430F1
:1001200027950D91043027950D9104302795A75000
:100130002695209528BB94DF93DF92DF0D91053043
:1001400027950D91053027950D91053027950D9137
:10015000053027950D91053027950D910530279590
:100160000D9105302795A7502695209528BB78DF5F
:1001700077DF76DF75DF0D91063027950D9106301C
:1001800027950D91063027950D91063027950D91F5
:10019000063027950D91063027950D91063027954D
:1001A000A7502695209528BB5BDF5ADF59DF58DF23
:1001B00057DF0D91073027950D91073027950D9149
:1001C000073027950D91073027950D91073027951A
:1001D0000D91073027950D9107302795A75026954B
:1001E000209528BB3DDF3CDF3BDF3ADF39DF38DFDE
:1001F0000D91083027950D91083027950D91083005
:1002000027950D91083027950D91083027950D9170
:10021000083027950D9108302795A75026952095F1
:1002200028BB1EDF1DDF1CDF1BDF1ADF19DF18DF15
:100230000D91093027950D91093027950D910930C1
:1002400027950D91093027950D91093027950D912E
:10025000093027950D9109302795A75026952095AF
:1002600028BBFEDEFDDEFCDEFBDEFADEF9DEF8DEBC
:10027000F7DE0D910A3027950D910A3027950D91E3
:100280000A3027950D910A3027950D910A30279550
:100290000D910A3027950D910A302795A750269584
:1002A000209528BBDDDEDCDEDBDEDADED9DED8DE63
:1002B000D7DED6DED5DE0D910B3027950D910B30B4
:1002C00027950D910B3027950D910B3027950D91AA
:1002D0000B3027950D910B3027950D910B302795FD
:1002E000A7502695209528BBBBDEBADEB9DEB8DE66
:1002F000B7DEB6DEB5DEB4DEB3DEB2DE0D910C30B5
:1003000027950D910C3027950D910C3027950D9167
:100310000C3027950D910C3027950D910C302795B9
:100320000D910C302795A7502695209528BB98DE77
:1003300097DE96DE95DE94DE93DE92DE91DE90DE31
:100340008FDE8EDE0D910D3027950D910D302795A6
:100350000D910D3027950D910D3027950D910D3094
:1003600027950D910D3027950D910D302795A750AC
:100370002695209528BB74DE73DE72DE71DE70DE9A
:100380006FDE6EDE6DDE6CDE6BDE6ADE69DE0D91C9
:100390000E3027950D910E3027950D910E30279533
:1003A0000D910E3027950D910E3027950D910E3041
:1003B00027950D910E302795A7502695209528BB9F
:1003C0004FDE4EDE4DDE4CDE4BDE4ADE49DE48DEE1
:1003D00047DE46DE45DE44DE43DE0D910F302795D5
:1003E0000D910F3027950D910F3027950D910F30FE
:1003F00027950D910F3027950D910F3027950D9171
:100400000F302795A7502695209528BB29DE28DE9A
:1004100027DE26DE25DE24DE23DE22DE21DE20DED0
:100420001FDE1EDE1DDE1CDE0AE00A95F1F700E885
:1004300008BB0895A895A0E611E0012F00950F7361
:10044000006402BB11DEA95F110F1034B1F70895EB
:100450000F931F932F93EEDF2F911F910F910A950A
:10046000B9F70895A0E600270D93AA38E9F7089593
:10047000A0E62D93AA38E9F708951A3218F4A0E6F9
:10048000A10F2C930895183370F4A1E6A10F2FE06B
:100490001A3220F0012F0952A01B201B2E93A036E8
:1004A00011F02A95D9F70895183378F4A1E6A10F31
:1004B00021E01A3220F0012F0952A01B200F2E93A9
:1004C000A03619F023952031D1F7089520E0D0DF30
:1004D00004E6BEDF2FE0CCDF04E6BADF089520E0BB
:1004E000C7DF0AE0B5DF23952F30D1F7C1DF0AE07F
:1004F000AFDF2A952F3FD1F70895B4DF2FE010E04A
:10050000BCDF1E5F1A32E0F308E2A2DFABDF2FE0B0
:1005100011E0B3DF1E5F1A32E0F308E299DF0895BD
:1005200020E010E0AADF13950FE020271A32D0F365
:100530000AE08EDF23952031A0F32FE010E09DDF4D
:1005400013950FE020271A32D0F30AE081DF2A95B5
:100550002031A0F308951FEF85DF2FE08EDF0AE042
:1005600077DF13951B32C1F708951AE27BDF2FE086
:1005700084DF0AE06DDF1A951F3FC1F708951FEF72
:1005800071DF81DF0AE064DF13951933C9F708953D
:1005900018E368DF89DF0AE05BDF1A951E3FC9F7C1
:1005A000089520E0869921E0303081F4213071F403
:1005B000E1990CC000E00CBB00E00EBB012F0095E0
:1005C0000295007F012B0DBBE29AE19A322F08952C
:1005D000A8953FEF00E00EBBE09A1DB3012F0095F8
:1005E0000295101789F41F70103079F0113099F0CE
:1005F0001230B9F0133011F1143031F1153049F1E6
:10060000163069F1173099F1A89560DF5FDF10E0CF
:10061000C8DF3130D1F3B3DFB2DF11E0C2DF3130F8
:10062000D1F36BDF6ADF69DF68DF67DF66DF65DF15
:1006300064DF63DF12E0B5DF313099F396DF95DFD9
:1006400013E0AFDF3130D1F34ADF14E0AADF3130FD
:10065000D9F39EDF9DDF15E0A4DF3130D1F360DFF9
:100660005FDF5EDF5DDF16E09CDF3130C1F373DFFB
:0C06700072DF17E096DF3130D1F3C6CF07
:00000001FF
